:100000000C9450010C941B0B0C94F40A0C94780182
:100010000C9478010C94A50D0C9478010C94770D38
:100020000C94B90C0C9478010C9478010C94780120
:100030000C9478010C9478010C9478010C9478015C
:100040000C94AA0A0C9478010C94680B0C94420B43
:100050000C9478010C9478010C9478010C9478013C
:100060000C949A0B0C94780168031801726818803C
:10007000234020035452414E534D495404035478B5
:10008000042020202020B55004B03B805F5004683D
:100090003B0205680576380A01285004683B282F82
:1000A0006805183802004F680576380A00295004A0
:1000B000683B212650046832101E50046832111F1C
:1000C000C004BF1103696804800200EE8003680168
:1000D000EA1804FF0200E16804C00200AEC0036831
:1000E00001AA681880234020035354414E444259CA
:1000F0002004032020042020202020E468188023EE
:100100004020032041555820492F5004032020044B
:100110002020202020E968188023402003432E203F
:10012000446973632004032020042020202020C37E
:1001300068188023402003425420417564696F048D
:10014000032020042020202020F368188023402052
:1001500003555342617564696F0403202004202015
:10016000202020A168188023402003464D20426EA5
:1001700064203304032020042020202020E368187A
:100180008023402003464D20626E64203204032009
:1001900020042020202020C268188023402003460D
:1001A0004D20626E64203104032020042020202092
:1001B00020C16818802340200344414220626E64BD
:1001C0003104032020042020202020AD6818802343
:1001D000402003414D20426E64203104032020045E
:1001E0002020202020E6681880234020034441423C
:1001F00020626E643304032020042020202020AFDE
:100200006818802340200344414220626E64320417
:10021000032020042020202020AE68051838030089
:100220004E68057638030020180A68390209003F35
:10023000000101776805183801004C6804BF02010D
:10024000D000000000240027002A00000000002544
:100250000028002B00000000080002010000030439
:10026000070000000000000000000000002300263E
:10027000002900040404040404040402020202022B
:10028000020303030303030102040810204080015A
:10029000020408102001020408102000040E7A1342
:1002A00011241FBECFEFD8E0DEBFCDBF24E0A0E712
:1002B000B1E001C01D92AB3BB207E1F711E0A0E055
:1002C000B1E0EAE0FAE202C005900D92A037B10772
:1002D000D9F711E0CFE4D1E004C02197FE010E94DC
:1002E000BD13CE34D107C9F70E94E20E0C94F81466
:1002F0000C940000833081F028F4813099F0823032
:10030000A9F008958730A9F08830C9F08430B1F49D
:10031000809180008F7D03C0809180008F778093D3
:100320008000089584B58F7784BD089584B58F7D4E
:10033000FBCF8091B0008F778093B00008958091BB
:10034000B0008F7DF9CFCF93DF93282F30E0F901F4
:10035000EB5AFD4F8491F901E957FD4FD491F90112
:10036000ED58FD4FC491CC23A1F081110E947A0178
:10037000EC2FF0E0EE0FFF1FE759FD4FA591B49170
:10038000EC91ED2381E090E009F480E0DF91CF91E2
:10039000089580E090E0FACF1F93CF93DF93282F4A
:1003A00030E0F901EB5AFD4F8491F901E957FD4F17
:1003B000D491F901ED58FD4FC491CC23A9F0162F2B
:1003C00081110E947A01EC2FF0E0EE0FFF1FE55B38
:1003D000FD4FA591B4918FB7F894EC91111108C01D
:1003E000D095DE23DC938FBFDF91CF911F910895CD
:1003F000DE2BF8CFCF93DF9390E0FC01E957FD4F60
:1004000024918D589D4FFC0184918823C9F090E080
:10041000880F991FFC01EF5BFD4FA591B491FC0182
:10042000E55BFD4FC591D49161110DC09FB7F89464
:100430008C91209582238C938881282328839FBFC9
:10044000DF91CF910895623051F49FB7F8943C91B9
:10045000822F809583238C93E8812E2BEFCF8FB74B
:10046000F894EC912E2B2C938FBFEACF3FB7F894E2
:100470008091400290914102A0914202B0914302CA
:1004800026B5A89B05C02F3F19F00196A11DB11DEF
:100490003FBFBA2FA92F982F8827BC01CD01620F2B
:1004A000711D811D911D42E0660F771F881F991FE6
:1004B0004A95D1F708952FB7F89460913C02709156
:1004C0003D0280913E0290913F022FBF0895089512
:1004D000089508950895AF92BF92CF92DF92EF9260
:1004E000FF920F931F93CF93DF936C017B018B01DE
:1004F000040F151FEB015E01AE18BF08C017D1072E
:1005000059F06991D601ED91FC910190F081E02DB7
:10051000C6010995892B79F7C501DF91CF911F910C
:100520000F91FF90EF90DF90CF90BF90AF90089524
:10053000FC01538D448D252F30E0842F90E0821BE9
:10054000930B541710F0CF96089501970895FC016E
:10055000918D828D981761F0A28DAE0FBF2FB11DC6
:100560005D968C91928D9F5F9F73928F90E008951E
:100570008FEF9FEF0895FC01918D828D981731F0D8
:10058000828DE80FF11D858D90E008958FEF9FEF2C
:100590000895FC01918D228D892F90E0805C9F4F02
:1005A000821B91098F739927089584E492E00E9439
:1005B000C90221E0892B09F420E0822F089580E010
:1005C00090E0892B29F00E94D50281110C94000043
:1005D0000895FC01A48DA80FB92FB11DA35ABF4FD8
:1005E0002C91848D90E001968F739927848FA68932
:1005F000B7892C93A089B1898C91837080648C9386
:10060000938D848D981306C00288F389E02D808134
:100610008F7D80830895EF92FF920F931F93CF9366
:10062000DF93EC0181E0888F9B8D8C8D98131AC02D
:10063000E889F989808185FF15C09FB7F894EE8914
:10064000FF896083E889F989808183708064808371
:100650009FBF81E090E0DF91CF911F910F91FF90BC
:10066000EF900895F62E0B8D10E00F5F1F4F0F7364
:100670001127E02E8C8D8E110CC00FB607FCFACF1F
:10068000E889F989808185FFF5CFCE010E94E902D2
:10069000F1CFEB8DEC0FFD2FF11DE35AFF4FF082F0
:1006A0009FB7F8940B8FEA89FB8980818062CFCF56
:1006B000CF93DF93EC01888D8823B9F0AA89BB8999
:1006C000E889F9898C9185FD03C0808186FD0DC084
:1006D0000FB607FCF7CF8C9185FFF2CF808185FFA5
:1006E000EDCFCE010E94E902E9CFDF91CF910895CD
:1006F0002091C001260F3327331F21323105ECF43E
:1007000020910F02FC0190E080E0243069F082E04B
:100710000895A091C0012191AC0140565E4FA40FF5
:10072000B52FB11D2C930196861798F38091C001C7
:10073000680F6093C00180E0089581E008951092F1
:100740000F0281E080930E021092E90161E082E1E4
:100750000E94CC0161E083E10E94CC01E9EBF0E072
:1007600080818E7F808380818D7F808388E48093E9
:10077000B80085E48093BC000895CF93DF9391E0A7
:1007800090939F018823B9F0C091B800D091BA002E
:100790008091BC008A7B8093BC0060E082E10E9473
:1007A000CC0160E083E10E94CC010E949F03D093C2
:1007B000BA00C093B800DF91CF9108950895E091F9
:1007C000E8018091E701E81730F4F0E0E158FE4FCE
:1007D000808190E008958FEF9FEF08959091E80158
:1007E0008091E7012FEF3FEF981748F4E92FF0E0F1
:1007F000E158FE4F208130E09F5F9093E801C901EE
:1008000008958091E7019091E801891B990B089563
:10081000CF92DF92EF92FF920F931F93CF93DF93CC
:100820007C01CB018A0120911502222389F0EB0182
:100830006B01C40ED51ECC15DD0569F06991D70199
:10084000ED91FC910190F081E02DC7010995F3CF66
:10085000642F0E947803C801DF91CF911F910F91FF
:10086000FF90EF90DF90CF900895CF93DF931F928A
:10087000CDB7DEB76983209115022223F9F02091CC
:100880003802203258F021E030E0FC01338322832B
:1008900090E080E00F90DF91CF9108958091160253
:1008A000E82FF0E0E95EFD4F998190838F5F8093A0
:1008B00016028093380281E090E0ECCF61E0CE0137
:1008C00001960E947803F7CF90E080E008958F9220
:1008D0009F92AF92BF92CF92DF92EF92FF924B0125
:1008E0005C010E9436026B017C0124E0C21AD1082F
:1008F000E108F1080E9436026C197D098E099F09F2
:10090000681579058A059B05A8F3FF90EF90DF90A5
:10091000CF90BF90AF909F908F900895FC018481FD
:100920009581228133812817390771F0860F971F2F
:10093000608171810E94A9130680F781E02DE80F84
:10094000F91F808190E008958FEF9FEF0895FC01DB
:1009500084819581228133812817390741F0860FE0
:10096000971F608171810E94A913958384830895E4
:10097000FC01462F22813381C9010196608171817A
:100980000E94A913648175818617970781F0A6815B
:10099000B781A20FB31F4C9382819381019660812E
:1009A00071810E94A9139383828380E008958FEF61
:1009B0000895EF92FF920F931F93CF93DF937C01E3
:1009C000062F10E0B8018DE194E00E94B804D0E059
:1009D000C0E0C017D10758F4F701EC0FFD1F649178
:1009E00070E08DE194E00E94B8042196F2CFDF918F
:1009F000CF911F910F91FF90EF90089580917E010C
:100A00008823B9F080917D01882399F06CE088E219
:100A100092E00E94D90467E081E292E00E94D9044A
:100A200067E08AE192E00E94D90461E08AE00C94D8
:100A3000CC0160E08AE00E94CC0167E084E392E0B0
:100A40000C94D904CF93DF93FC01C281D3818481BC
:100A50009581C817D907C9F0A681B781A80FB91F1A
:100A60002C910196608171810E94A913C817D90742
:100A700039F095838483822F90E0DF91CF910895A0
:100A80001582148213821282F6CF8FEF9FEFF5CF7B
:100A9000FC0160817181848195819B01281B390B48
:100AA00082819381820F931F0E94A9130895DC0114
:100AB000ED91FC910190F081E02D09948091D80393
:100AC000882319F060E00C94CC012D9808958823B8
:100AD00049F08091D803882319F061E00C94CC018F
:100AE0002D9A08950C945E05CF93DF93EB018091CE
:100AF000D903823019F481E00E9467052998BE016C
:100B000090E080E00E946704299A8091D9038230A6
:100B100031F40E945E05DF91CF910C945E05DF9168
:100B2000CF9108958F929F92AF92BF92CF92DF9212
:100B3000EF92FF921F93CF93DF93EC014A015B0189
:100B4000219A8FEF88169806A806B806E1F4219A34
:100B500060E073E2CE010E94740560EC78E080E012
:100B600090E00E94670460E372E0CE01DF91CF91D4
:100B70001F91FF90EF90DF90CF90BF90AF909F902C
:100B80008F900C94740560E073E2CE010E947405AE
:100B900060E871E180E090E00E94670410E2C12CFF
:100BA000D12CE12C90E8F92ED501C4018C219D2196
:100BB000AE21BF2160E372E0892B8A2B8B2B81F061
:100BC000CE010E94740560E976E080E090E00E942A
:100BD0006704F694E794D794C794115029F7C3CFCC
:100BE000CE010E94740560E372E080E090E0EFCFF8
:100BF000CF9327E734E0F90101900020E9F79F0146
:100C000028573440C091720433274C2F50E0BA016A
:100C100061507109261B370B30936D0420936C04CF
:100C2000682F70E069587B4F84E191E00E94E814DE
:100C300080911401803219F486E880931401CB5F0F
:100C4000C0930F01EC2FF0E0319620E090E0A92F47
:100C5000B0E0A25FBE4F4C9124279F5FC917B8F741
:100C6000E25FFE4F208360910F0170E06E5F7F4F67
:100C700085E294E00E94B804C0E02C2F30E080911F
:100C80000F0190E00196821793075CF0225F3E4FC0
:100C9000F901608170E085E294E00E94B804CF5FC2
:100CA000ECCFCF91089585ED8093BC008091110227
:100CB00090911202A0911302B09114020796A11D07
:100CC000B11D23E0B695A795979587952A95D1F7FD
:100CD0002091BC0024FD03C010920F0208954091A2
:100CE0001102509112026091130270911402452B6F
:100CF000462B472B69F30097A105B10541F02AE285
:100D00002A95F1F700C00197A109B109E1CF8091BF
:100D100010020C94BD031F93CF93DF93EC01162FA9
:100D20000E949313181739F0612FCE01DF91CF91F4
:100D30001F910C949B13DF91CF911F9108950C94F8
:100D400093138BE090E00E949F06282F30E03093B1
:100D5000090120930801823071F018F4813031F0DC
:100D60000895833061F0843071F008956AE182EB78
:100D700091E00C94D9046AE180E092E0FACF6AE154
:100D800086EE91E0F6CF6AE18CEC91E0F2CFCF9362
:100D9000DF9390E080E00E949F06C82FD0E0D093C0
:100DA0000701C09306018AE090E00E949F06282F69
:100DB00030E03093050120930401C130D10559F48E
:100DC000823011F1833021F1813029F46AE182EB24
:100DD00091E00E94D9048AE090E00E949F06282FAB
:100DE00030E030930501209304012297E9F482302A
:100DF00099F08330A9F08130B9F46AE188E991E093
:100E0000DF91CF910C94D9046AE180E092E0E1CFC8
:100E10006AE186EE91E0DDCF6AE18EE791E0F0CF06
:100E20006AE184E691E0ECCFDF91CF91089590E004
:100E300080E00E949F06282F30E03093030120932A
:100E400002018150873008F047C0E82FF0E0E55DEF
:100E5000F84F0C94BD133207380743074C0755076A
:100E60005907620710927D010E94FE040C94A106AE
:100E700010927D010E94FE046AE188E991E00E94DF
:100E8000D9040C94C70610927D010E94FE046AE109
:100E90008AE491E00C94D9046AE180E391E00E9435
:100EA000D90410927D010C94FE046AE186E191E080
:100EB000F6CF6AE18CEF90E00E94D90481E0809344
:100EC0007D01F1CF10927D010E94FE046AE182EE65
:100ED00090E00E94D904E7CF08958F929F92AF923D
:100EE000BF92CF92DF92EF92FF920F931F93CF9317
:100EF000DF93CDB7DEB768970FB6F894DEBF0FBEAD
:100F0000CDBF7C01FC010081C280D38016810E948C
:100F10005B028090700190907101A0907201B0907E
:100F200073019B01AC01281939094A095B09490180
:100F30005A0130E1831637E29306A104B10468F048
:100F400060937001709371018093720190937301AB
:100F500065E088E690E00E94D90445E050E06DED40
:100F600070E0C7010E948613892B29F466E087EDA3
:100F700090E00E94D90446E050E061ED70E0C701C6
:100F80000E948613892B19F481E080937E01809161
:100F90003A0281110AC066E08BE392E00E94D90414
:100FA0000E94170781E080933A0245E050E06CEC24
:100FB00070E0C7010E948613892B29F466E086EC55
:100FC00090E00E94D90445E050E060EC70E0C70179
:100FD0000E948613892B11F40E941707003809F02C
:100FE00090C24FEBC41290C258E1D5128DC261E09D
:100FF00081E10E94CC0180917C01811105C00E9499
:10100000170781E080937C0168960FB6F894DEBFE5
:101010000FBECDBFDF91CF911F910F91FF90EF9049
:10102000DF90CF90BF90AF909F908F900895153034
:1010300009F4D6C0163041F766E08AE990E00E94D4
:10104000D90480917D01882309F403C180917E0138
:10105000882309F4FEC067E083E990E0DBC01A3022
:1010600009F472C108F040C0183009F4F7C0193013
:1010700059F690E080E00E949F0690E0909307016F
:1010800080930601019709F022C14FE450EB62E61C
:101090007DE988E791E00E94920580910801909196
:1010A00009010196843091050CF00EC1909309015D
:1010B00080930801609108018BE090E00E948B060C
:1010C00068960FB6F894DEBF0FBECDBFDF91CF910B
:1010D0001F910F91FF90EF90DF90CF90BF90AF9056
:1010E0009F908F900C94A1061B3009F46EC11C30A8
:1010F00009F08ACF66E087E890E00E94D90447E1D2
:1011000058EE62E67DE922C01A3209F496C1A0F5D4
:10111000173209F4CAC180F4163209F075CF8091F4
:101120007D01882321F080917E01811175C04FE6F9
:1011300050E962E67DE90AC0183209F4C3C14FE9FB
:1011400050E662E67DE9193209F05ECF88E791E06A
:1011500068960FB6F894DEBF0FBECDBFDF91CF917A
:101160001F910F91FF90EF90DF90CF90BF90AF90C5
:101170009F908F900C9492051D3209F468C150F431
:101180001B3209F45FC14FE350EC62E67DE91C328B
:10119000E9F23ACF1E3209F483C11E3409F034CF8C
:1011A00060E08AE068960FB6F894DEBF0FBECDBF50
:1011B000DF91CF911F910F91FF90EF90DF90CF9033
:1011C000BF90AF909F908F900C94CC0166E08AEB1B
:1011D00090E00E94D90447ED58E262E67DE9B6CF7F
:1011E00066E084EB90E00E94D90447E558EA62E6A5
:1011F0007DE9ACCF66E08EEA90E00E94D904809150
:101200007D0167E08823E1F080917E018823C1F0B1
:1012100087EA90E00E94D90468960FB6F894DEBF82
:101220000FBECDBFDF91CF911F910F91FF90EF9037
:10123000DF90CF90BF90AF909F908F900C94FE0462
:1012400080EA90E00E94D9044FE850E762E67DE929
:101250007DCF4FEA50E562E67DE978CF66E08DE824
:1012600090E00E94D90447EC58E362E67DE988E704
:1012700091E00E94920580910201909103010196F4
:1012800088309105F4F490930301809302016091FA
:10129000020190E080E00E948B0668960FB6F894F9
:1012A000DEBF0FBECDBFDF91CF911F910F91FF9099
:1012B000EF90DF90CF90BF90AF909F908F900C9465
:1012C000170781E090E0DFCF81E090E0EFCE90E083
:1012D00080E00E949F0690E09093070180930601B2
:1012E000029709F091CE4FE450EB62E67DE988E782
:1012F00091E00E9492058091040190910501019670
:1013000084309105F4F49093050180930401609179
:1013100004018AE090E00E948B0668960FB6F8946C
:10132000DEBF0FBECDBFDF91CF911F910F91FF9018
:10133000EF90DF90CF90BF90AF909F908F900C94E4
:10134000C70681E090E0DFCF80910001909101011C
:10135000019686309105A4F59093010180930001D8
:10136000609100018CE890E00E948B068CE890E090
:101370000E949F0690E0909301018093000128E174
:10138000E4E3F1E0DE01119601900D922A95E1F778
:10139000880F991F880F991FE1E0F0E0EC0FFD1F07
:1013A0008E0F9F1FFC01408151816281738184E710
:1013B00091E00E9492054FEC50E362E67DE9C6CED3
:1013C0001092010110920001CBCF4EE251ED62E686
:1013D0007DE9BCCE61E08AE00E94CC018CE00E94F5
:1013E000A301892B39F060E08CE00E94CC010E94BF
:1013F0001707A3C061E08CE00E94CC0147E958E6E2
:1014000062E67DE988E791E00E9492056AE18DE657
:1014100090E068960FB6F894DEBF0FBECDBFDF91A7
:10142000CF911F910F91FF90EF90DF90CF90BF90E1
:10143000AF909F908F900C94D9044FE750E862E6EC
:101440007DE984CE46EB59E462E67DE97FCE4EE34A
:1014500051EC62E67DE988E791E00E94920561E047
:1014600090E080E00E948B0661E08AE090E00E94BC
:101470008B0661E08BE090E00E948B0660E08EE1DD
:1014800090E00E948B0660E088E290E00E948B066C
:1014900060E08CE890E00E948B060E9417073DCF29
:1014A0004FE550EA62E67DE951CE80917D018823C7
:1014B00021F080917E018111AFCE4FE150EE62E6C6
:1014C0007DE944CE4FEE50E162E67DE988E791E0A8
:1014D0000E94920562E090E080E068960FB6F89472
:1014E000DEBF0FBECDBFDF91CF911F910F91FF9057
:1014F000EF90DF90CF90BF90AF909F908F900C9423
:101500008B06003C09F080CDF1E3DF127DCD61E078
:1015100085E00E94CC011E3009F45CCF08F0F4CDC8
:10152000173009F467CE08F09ACD143009F44ECE86
:1015300008F07DCD133009F067CD47E958E662E643
:101540007DE904CEFC0186819781009711F00C940F
:101550005F1408951F920F920FB60F9211242F93CC
:101560003F938F939F93AF93BF9380913C02909151
:101570003D02A0913E02B0913F0230913B0223E038
:10158000230F2D3758F50196A11DB11D20933B0265
:1015900080933C0290933D02A0933E02B0933F02A1
:1015A0008091400290914102A0914202B091430289
:1015B0000196A11DB11D8093400290934102A0931A
:1015C0004202B0934302BF91AF919F918F913F919F
:1015D0002F910F900FBE0F901F90189526E8230FA4
:1015E0000296A11DB11DD2CF1F920F920FB60F927E
:1015F00011242F933F934F935F936F937F938F9318
:101600009F93AF93BF93EF93FF93E0910C01F09101
:101610000D010995FF91EF91BF91AF919F918F912E
:101620007F916F915F914F913F912F910F900FBEDE
:101630000F901F9018951F920F920FB60F921124C2
:101640002F933F934F935F936F937F938F939F93CA
:10165000AF93BF93EF93FF93E0910A01F0910B01D9
:101660000995FF91EF91BF91AF919F918F917F91DC
:101670006F915F914F913F912F910F900FBE0F90FF
:101680001F9018951F920F920FB60F9211242F934F
:101690003F934F935F936F937F938F939F93AF93FA
:1016A000BF93EF93FF9384E492E00E94E902FF91DD
:1016B000EF91BF91AF919F918F917F916F915F91CA
:1016C0004F913F912F910F900FBE0F901F90189543
:1016D0001F920F920FB60F9211242F938F939F9307
:1016E000EF93FF93E0915402F09155028081E091D5
:1016F0005A02F0915B0282FD1BC0908180915D02D5
:101700008F5F8F7320915E02821741F0E0915D023E
:10171000F0E0EC5BFD4F958F80935D02FF91EF91C0
:101720009F918F912F910F900FBE0F901F90189542
:101730008081F4CF1F920F920FB60F9211242F9336
:101740003F934F935F936F937F938F939F93AF9349
:10175000BF93EF93FF938091B900887F803609F49F
:101760004AC0F0F5883209F4A7C018F5803109F4B1
:101770009BC0B8F4882309F4F9C0883009F494C0F8
:10178000FF91EF91BF91AF919F918F917F916F9159
:101790005F914F913F912F910F900FBE0F901F902F
:1017A0001895883109F488C0803251F780930D0272
:1017B00014C0803409F49DC040F48033B9F38833F9
:1017C000F9F680930D0285ECB0C0803509F485C030
:1017D000883509F496C0883499F60E945306D0CF14
:1017E000883909F48CC038F5883729F050F48836E8
:1017F00011F0803729F683E080930F021092E20106
:1018000057C0883809F47BC0803919F0803809F056
:10181000B7CF8091E201803208F071C0E091E2011F
:1018200081E08E0F8093E2018091BB00F0E0EE53E7
:10183000FE4F80833DC0803B39F0E0F4803A09F4EC
:1018400079C0883A09F09CCF84E080930F0210920F
:10185000C1011092C001E091E501F091E601099506
:101860008091C00181110FC081E08093C00110926E
:10187000A00109C0803C09F4A6CF883C09F4A3CF9D
:10188000883B09F07DCFE091C10181E08E0F80930C
:10189000C101F0E0E056FE4F80818093BB00909143
:1018A000C1018091C00129C08091EA018093BB00F1
:1018B00085EC8093BC0064CF90910C0280910B0268
:1018C000981758F5E0910C0281E08E0F80930C027E
:1018D000F0E0E551FE4F8081E9CFE0910C0281E01C
:1018E0008E0F80930C028091BB00F0E0E551FE4F1B
:1018F000808390910C0280910B029817C8F285E8C2
:10190000D8CFE0910C0281E08E0F80930C02809181
:10191000BB00F0E0E551FE4F808380910E02811103
:101920005CCF81E08093E90184EA8093BC0010924F
:101930000F0226CF85EC8093BC0010920F0280919D
:10194000E201803230F4E091E201F0E0EE53FE4F2C
:1019500010826091E20170E0E091E301F091E40116
:1019600082EC91E009951092E2010ACF10920D02EB
:1019700034CF1F920F920FB60F9211242F933F93E3
:101980004F935F936F937F938F939F93AF93BF9387
:10199000CF93EF93FF93E091EF02F091F002C081BB
:1019A0008091F102C8238091F2029091F302019696
:1019B00049F08091F2029091F30201969093F30224
:1019C0008093F2028091ED0281111DC0C1116EC0A1
:1019D0008091F2029091F302813A910578F0109291
:1019E000F6028091F2029091F3029093F9028093B3
:1019F000F80281E08093F7028093ED021092F302E7
:101A00001092F20253C08091ED028130A9F4CC23F0
:101A100009F44CC0E091F7028E0F8093F702809199
:101A2000F2029091F302F0E0EE0FFF1FE351FD4F41
:101A30009487838782E0E0CF8091ED02823009F0C5
:101A40004FC0C11122C0E091F70281E0E03768F099
:101A50008093F60283E08093ED02E091F402F0912E
:101A6000F502309759F20995C9CF8E0F8093F7028E
:101A70008091F2029091F302F0E0EE0FFF1FE3512C
:101A8000FD4F9487838781E0B7CF8091F2029091D8
:101A9000F302813A910550F083E08093ED02E091EA
:101AA000F402F091F502309709F009958091D9037D
:101AB000813021F4C11180E00E946705FF91EF9110
:101AC000CF91BF91AF919F918F917F916F915F91D6
:101AD0004F913F912F910F900FBE0F901F9018952F
:101AE0008091ED02833011F7C111E0CF87CF1F92B3
:101AF0000F920FB60F9211242F933F934F935F9342
:101B00006F937F938F939F93AF93BF93EF93FF93C5
:101B100081E08093390260E08DE00E94CC01E1EB2E
:101B2000F0E08081887F8083FF91EF91BF91AF913A
:101B30009F918F917F916F915F914F913F912F91E5
:101B40000F900FBE0F901F9018951F920F920FB617
:101B50000F9211242F933F934F935F936F937F9333
:101B60008F939F93AF93BF93EF93FF9380E00E9477
:101B7000A3010197D9F481E00E94A3010197B1F478
:101B80008091B10087608093B100FF91EF91BF9188
:101B9000AF919F918F917F916F915F914F913F9105
:101BA0002F910F900FBE0F901F90189580E00E940C
:101BB000A301892B51F781E00E94A301019729F726
:101BC0001092390261E08DE00E94CC018091B10059
:101BD000887FD9CF0F931F93CF93DF93EC018B01B5
:101BE000798368831D821C821B821A82CB010E942A
:101BF000C3139F838E83A80170E060E0DF91CF91D3
:101C00001F910F910C94F114CF93DF93E4E4F2E071
:101C10001382128288EE93E0A0E0B0E08483958383
:101C2000A683B78320E531E03183208325EC30E0C3
:101C30003587248724EC30E03787268720EC30E096
:101C4000318B208B21EC30E0338B228B22EC30E087
:101C5000358B248B26EC30E0378B268B118E128E41
:101C6000138E148EE1EEF2E0138212828483958348
:101C7000A683B78382E691E091838083EDEEF2E064
:101C8000F0930104E0930004118281E0848389E2EF
:101C900090E09383828350981092D803CDE2D4E0F1
:101CA0001CAA0E945B02609311047093120480933B
:101CB0001304909314040E945B0260930D047093CC
:101CC0000E0480930F049093100419861A861B86C5
:101CD00018861F821E821D8262E080E00E94FA0147
:101CE00061E084E00E94FA0161E084E00E94CC019E
:101CF000E0EBF0E010821092B1008DE98093B30028
:101D0000808182608083E0E7F0E080818260808370
:101D1000E8E6F0E0808184608083EDE6F0E0808199
:101D20008160808319821A8280ED97E09AAF89AF33
:101D300088EE93E09CAF8BAF88EC90E09EAF8DAFC8
:101D400082E08093730410926D0410926C048BE017
:101D500080937204109274041092750410927604A9
:101D60000E945B0260936E0470936F048093700412
:101D7000909371040E945B026093110470931204AB
:101D800080931304909314040E945B0260930D04EB
:101D900070930E0480930F049093100460E870E039
:101DA00085E194E00E94EA0D60E470E08DE194E04A
:101DB0000E94EA0D60E470E085E294E0DF91CF914B
:101DC0000C94EA0D789484B5826084BD84B58160FA
:101DD00084BD85B5826085BD85B5816085BD8091F6
:101DE0006E00816080936E0010928100809181006E
:101DF0008260809381008091810081608093810066
:101E0000809180008160809380008091B100846027
:101E10008093B1008091B00081608093B000809188
:101E20007A00846080937A0080917A008260809347
:101E30007A0080917A00816080937A0080917A00A4
:101E4000806880937A001092C10061E085E00E9472
:101E5000FA0161E086E00E94FA0160E08AE00E94F7
:101E6000FA0161E08BE00E94FA0161E08CE00E94DF
:101E7000FA0162E084E10E94FA0161E08DE00E94D3
:101E8000FA01E0915402F091550282E08083E091E2
:101E90005002F09151021082E0915202F0915302EF
:101EA00080E1808310925C02E0915802F091590227
:101EB00086E08083E0915602F09157028081806134
:101EC0008083E0915602F091570280818860808380
:101ED000E0915602F0915702808180688083E09102
:101EE0005602F091570280818F7D808361E085E00A
:101EF0000E94CC011092E8011092E70110921602A4
:101F0000109238020E949F0388E692E09093E601C7
:101F10008093E50189E692E09093E4018093E301E8
:101F200081E0809315028FE2809337026FE781EEA4
:101F300092E00E943504C0913802C13208F091C08D
:101F40000E9436026B017C0180910F02811164C0F6
:101F500082E080930F0281E080930E028FEF8093E6
:101F60000D0210920C02C0930B02A7E1B2E0EBEE5F
:101F7000F1E080E0C81323C11092EA018091EA01E8
:101F80008E658093EA018091E901813009F01BC1DF
:101F90001092E9010E9436026B017C018091EA01F6
:101FA0008093BB008091110290911202A0911302C4
:101FB000B0911402892B8A2B8B2B99F00E94360248
:101FC000009111021091120220911302309114021B
:101FD0006C197D098E099F0906171707280739070D
:101FE000E0F18091BC0083FDD9CF85EC8093BC00EB
:101FF0000E9436026B017C0180910F02823009F44D
:10200000E4C080910D028F3F61F180910D0280321A
:1020100041F180910D0225C0809111029091120230
:10202000A0911302B0911402892B8A2B8B2B09F4F7
:102030008BCF0E9436020091110210911202209162
:102040001302309114026C197D098E099F0906173D
:1020500017072807390708F077CF809110020E94F0
:10206000BD0310921602109238021092150284E4F9
:1020700092E09093310480933004E0915402F09107
:10208000550292E09083E0915002F091510210824B
:10209000E0915202F09153028FEC808310925C0227
:1020A000E0915802F091590286E28083E091560255
:1020B000F0915702808180618083E0915602F09117
:1020C0005702808188608083E0915602F091570228
:1020D000808180688083E0915602F0915702808170
:1020E0008F7D80832CED35E0309367042093660468
:1020F00028EE33E0309369042093680428EC30E044
:1021000030936B0420936A04909373048DE697E0F8
:10211000909365048093640461E08DE00E94FA016D
:1021200092E0292E312CEE24E394F12C34E0C32EDE
:10213000D12C80913A0281112FC00E9436024B01AE
:102140005C0188EE482E83E0582E612C712C0E9491
:102150003602681979098A099B09683E734081052E
:102160009105A8F321E0421A51086108710888EE30
:10217000880E83E0981EA11CB11C41145104610417
:10218000710429F766E08BE392E00E94D9040E9473
:102190001707B1E0B0933A02E0913204F0913304B2
:1021A000E830F105B0F5E952FF4E0C94BD1307116C
:1021B000C211D811FB11241239124D126E129D91C9
:1021C00091938F5FD7CE85EE11CF809111029091C0
:1021D0001202A0911302B0911402892B8A2B8B2B2F
:1021E00009F40ACF0E9436020091110210911202E6
:1021F00020911302309114026C197D098E099F09F8
:10220000061717072807390708F0F6CE26CF1092D1
:102210007404809139028823E1F085E294E00E9401
:10222000480518161906ACF485E294E00E942205D0
:10223000EC0180E00E94A301019731F4B12CA12CA4
:10224000C331D10508F470C1BE0185E294E00E945B
:10225000A7048091300490913104DC01ED91FC9150
:102260000084F185E02D0995892B81F0809130045F
:1022700090913104DC01ED91FC910284F385E02D15
:102280000995BC0185E194E00E94B8048091340472
:10229000909135048230910509F49BC108F058C132
:1022A000009709F463C1019709F475C1809139025F
:1022B0008823C9F18DE194E00E944805181619069B
:1022C00094F50E945B0200910D0410910E04209180
:1022D0000F0430911004601B710B820B930B6A305A
:1022E000710581059105F8F08DE194E00E942205C9
:1022F000EC0180E00E94A301019731F4B12CA12CE4
:10230000C132D1050CF4E2C1BE018DE194E00E941E
:10231000A7040E945B0260930D0470930E048093E7
:102320000F049093100480912E04882371F00E9472
:102330005B0260E084E00E94CC0170E060E080918C
:102340003004909131040E9457050E945B02613471
:102350007F418105910548F08BE00E94A301019720
:1023600021F460E08BE00E94CC0180E090E0892BBA
:1023700009F4DFCE0E94D502882309F4DACE0E9448
:102380000000D7CE109276041092750480E00E946F
:10239000F80530923304209232040E945B0260936D
:1023A0006E0470936F04809370049093710431CF26
:1023B0000E945B0200916E0410916F0420917004E2
:1023C00030917104AB01BC01401B510B620B730BCC
:1023D0008091660490916704B0E0A0E04817590727
:1023E0006A077B0708F415CF83E090E090933304ED
:1023F000809332040ECF8091750420916C0430914B
:102400006D048217130680F48F5F809375048091AA
:10241000760491E0980F909376040E94F805D0928C
:102420003304C0923204B9CFA5E0B0E0B0933304D6
:10243000A093320410927604109275048091740473
:102440008F5F80937404E5CE0E945B0200916E045E
:1024500010916F042091700430917104AB01BC01A4
:10246000401B510B620B730B80916A0490916B04BB
:10247000B3CF9091740480917304981738F486E078
:1024800090E0909333048093320487CFA7E0B0E0CC
:10249000B0933304A093320480CF0E945B0200917A
:1024A0006E0410916F042091700430917104AB019F
:1024B000BC01401B510B620B730B8091680490911F
:1024C0006904B0E0A0E0481759076A077B0708F4E1
:1024D000A0CEF0923304E09232049BCE0E945B02C5
:1024E00000916E0410916F0420917004309171047A
:1024F000AB01BC01401B510B620B730B8091680454
:1025000090916904B0E0A0E0481759076A077B077B
:1025100008F47FCE1092760480E00E94F8051092B5
:1025200033041092320475CE0091300410913104BE
:10253000CA15DB0509F48DCE85E294E00E942205E0
:10254000BC01C8010E945705BFEFAB1ABB0AECCF14
:102550008330910509F477C061E070E0049709F0D9
:10256000A5CE85E194E00E94A704ABC085E194E08C
:102570000E944805181619060CF098CE70E060E02D
:1025800085E194E00E948E0480933604F092350435
:10259000E09234048BCE85E194E00E9448050297D6
:1025A0000CF484CE61E070E085E194E00E948E043A
:1025B000809337048350823228F43092350420927D
:1025C000340474CE61E070E085E194E00E94A704D9
:1025D0006DCE0091370410E05801BFEFAB1ABB0A73
:1025E00085E194E00E944805A816B9060CF05ECE7D
:1025F000712CD0E0C0E0BE0185E194E00E948E0421
:10260000782621960C171D07B4F7B50185E194E0F3
:102610000E948E047816190689F40E945B0260936A
:10262000110470931204809313049093140483E0B4
:1026300090E0909335048093340438CED0923504E2
:10264000C092340433CE80913604982F9F77903512
:1026500021F0982F9F7B903899F4CDE2D4E09E0131
:102660002D52344021968091370490E001968217D4
:102670009307ECF085E194E00E9422058B87EFCF71
:10268000893759F3982F9D7F983639F38F3329F383
:10269000883119F3982F9F7D983CF9F260913704A7
:1026A00070E06E5F7F4F803B09F05BCFD6CF91E04B
:1026B00090936104E0916404F091650489E394E0EF
:1026C00009951092350410923404F0CDAC16BD0675
:1026D0000CF01FCE00913004109131048DE194E094
:1026E0000E942205BC01C8010E945705AFEFAA1A3B
:1026F000BA0AECCF85E294E00E94A20A8DE194E050
:102700000E94A20A85E194E00C94A20AFB01DC017C
:1027100004C08D910590801921F441505040C8F7B4
:10272000881B990B0895F999FECF92BD81BDF89A47
:10273000992780B50895262FF999FECF1FBA92BD2B
:1027400081BD20BD0FB6F894FA9AF99A0FBE019692
:102750000895AA1BBB1B51E107C0AA1FBB1FA617E8
:10276000B70710F0A61BB70B881F991F5A95A9F73A
:1027700080959095BC01CD010895EE0FFF1F059047
:10278000F491E02D09940F931F93CF93DF93823040
:10279000910510F482E090E0E091B904F091BA0460
:1027A00030E020E0B0E0A0E0309799F42115310549
:1027B00009F44AC0281B390B24303105D8F58A8129
:1027C0009B816115710589F1FB0193838283FE0171
:1027D00011C0408151810281138148175907E0F0EF
:1027E0004817590799F4109761F012960C931297B5
:1027F00013961C933296CF01DF91CF911F910F91C9
:1028000008950093B9041093BA04F4CF211531054B
:1028100051F04217530738F0A901DB019A01BD01BD
:10282000DF01F801C1CFEF01F9CF9093BA04809393
:10283000B904CDCFFE01E20FF31F81939193225093
:10284000310939832883D7CF2091B7043091B80458
:10285000232B41F420913001309131013093B804A1
:102860002093B70420912E0130912F0121153105BD
:1028700041F42DB73EB74091320150913301241BF2
:10288000350BE091B704F091B804E217F307A0F418
:102890002E1B3F0B2817390778F0AC014E5F5F4FB6
:1028A0002417350748F04E0F5F1F5093B80440932C
:1028B000B704819391939FCFF0E0E0E09CCFCF935A
:1028C000DF930097E9F0FC01329713821282A09106
:1028D000B904B091BA04ED0130E020E01097A1F402
:1028E00020813181820F931F2091B7043091B80469
:1028F0002817390709F061C0F093B804E093B704D2
:10290000DF91CF910895EA01CE17DF07E8F54A81FC
:102910005B819E0141155105B1F7E901FB83EA8313
:1029200049915991C40FD51FEC17FD0761F48081BF
:1029300091810296840F951FE90199838883828192
:1029400093819B838A83F0E0E0E012968D919C91C5
:1029500013970097B9F52D913C911197CD010296EF
:10296000820F931F2091B7043091B80428173907BC
:1029700039F6309751F51092BA041092B904B09319
:10298000B804A093B704BCCFD383C28340815181E4
:10299000840F951FC817D90761F44E5F5F4F888178
:1029A0009981480F591F518340838A819B8193836A
:1029B00082832115310509F0B0CFF093BA04E0937A
:1029C000B9049ECFFD01DC01C0CF13821282D7CFA4
:1029D000FB01DC0102C001900D9241505040D8F73C
:1029E0000895DC0101C06D9341505040E0F7089517
:1029F00011E0CFE4D1E004C0FE010E94BD13219696
:0A2A0000C035D107C9F7F894FFCFE5
:102A0A00010001000100010001006A026A02C80017
:102A1A008023423200000000000000000000000095
:102A2A00000000000000000000000000000000009C
:102A3A00BB0480007F80629DBF40629D3FC0629D53
:102A4A00DF20629D5FA0629D9F60629D0000000082
:102A5A000B036B0298025803C902A702BB020000CB
:102A6A000000350408046404DE030104EE03DF03F6
:00000001FF
